:03000000120003E8
:0300330002005276
:1019820019E319E71A091A271A3D1A4F1A591A6345
:0319920000000052
:10000300E4F5D0C2AF75818F12001675D0001213BC
:030013007180FEFB
:0C00160090198278087E197F95121979E4
:0100220022BB
:1019950012010101FF0000401D0700103000010287
:1019A500030109023C00010104802B090400000623
:1019B500FF0000050705010240000107050202407E
:1019C50000010705030240000107058102400001EF
:1019D5000705820240000107058302400001040358
:1019E500090422034500690063006F006E002000B2
:1019F50054006500630068006E006F006C006F00A6
:101A0500670079001E034500690063006F006E00E2
:101A150020004400490056004100200055005300B5
:101A2500420016033C002D002D0053006500720096
:101A350023002D002D003E001203530074006100A9
:101A45006E0064006100720064000A0349005000E2
:101A5500410043000A033000300037003900040319
:101A65003F00020D37020DDC020D3D020D52020D45
:101A75006A020D76020D7F020D8D020D99020DA6EB
:101A8500020DCE020DD5800000000000020001818C
:101A95000000000000020002820000006500020054
:101AA5000302030000650000000502010000650057
:101AB5000000078006000100007878088006000213
:101AC500000078780980067303787878780A8008AA
:101AD5000000000001000B00096E00000000000C72
:101AE500810A0000000001000D40E06E006C6800F6
:101AF500000FC0E100006C6801001001184F0315CC
:101B0500A80215EC0515FE0716580816910916A624
:101B15000A16BB0B17930C17A20D17B40E17C30F9C
:051B250017D51017F6B2
:0E002300ED1D6009EF0FF97700ED1D70F7225B
:100036007C05EC600D7DC6ED60041DED70FC1CECCE
:1000460070F31FBFFF011EEE4F70E522C0D053D8DC
:10005600EFD0D032907FA5E054406008907FA5E0B5
:10006600544070F8907FA57480F022907FA574406C
:10007600F022907FA6EFF0907FA5E05401700890E3
:100086007FA5E0540160F822907FA5E05401700836
:10009600907FA5E0540160F8907FA6E0228E1F8F26
:1000A600208D2112005A7FA2120078AF1F1200780D
:1000B600AF20120078AF2112007812007112005A98
:1000C6007FA2120078120071907FA5E0540260EDC5
:1000D600228E228F2312005A7FA2120078AF22129C
:1000E6000078AF2312007812007112005A7FA31213
:1000F6000078907FA57420F012008E12008EF524F1
:10010600120071E52422901B3EEFF0901B3FEDF0AC
:10011600907FE3741BF0907FE4743EF0907F98E04C
:1001260054EFF0907FE5E0907F98E04410F0907FE8
:10013600E5E022901B3EEFF0907FE3741BF0907F8A
:10014600E4743EF0907F98E054EFF0907FE5E0FF96
:10015600907F98E04410F0907FE5EFF0901B3FE031
:10016600228F25852518E51B700FE525F45407C455
:100176000354F8FD7FC512010C907F98E04402F00D
:10018600740455186007907F98E054FDF0228F267E
:100196008D27E527600EAA2674010A1333C3DAFCFD
:1001A6004218800DAA2674010A1333C3DAFCF452EE
:1001B60018AF18120167228F828E83E0FAEF2401AE
:1001C600F582E43EF583E0C39A228F828E83E0FABD
:1001D60004F0EF2402F9E43EF8E92AF582E438F562
:1001E60083E0228F828E83E02DFAEF2402F9E43E2B
:1001F600F8E92AF582E438F583E022EF2401F58256
:10020600E43EF583E08F828E83FAE0C39A1422AB34
:1002160005EF2401F582E43EF583E0FA04F0EF24CD
:1002260002F9E43EF8E92AF582E438F583EBF02298
:100236008F828E83E02DF0228F2B8D2C8B2D7F4885
:100246007E2512020124AD50667D027F487E25126E
:1002560002157DFF7F487E2512021590264EE0FD91
:100266007F487E251202157D077F487E25120215DE
:10027600AD8C7F487E25120215AD2B7F487E251258
:100286000215AD2C7F487E25120215AD2D7F487EC6
:1002960025120215AD287F487E25120215AD297F4D
:1002A600487E25120215AD2A7F487E25120215903A
:1002B600264EE004F0228F2E8D2F7480652E601856
:1002C6007421452EFF1201395404600C7421452E09
:1002D600FF120139540470F4AD2F7421452EFF121C
:1002E600010C227D207FC912010C7F067E001200C0
:1002F600367D007FC912010C7D107FCA12010C7D6C
:10030600387FC412010C7DC77FC412010C7D2F7F7C
:100316002012010C7D2F7F6012010C7D2A7FA01216
:10032600010C7DD57FC112010C228D308B317FB03F
:10033600120139F532E53014600614603A0203B34F
:10034600E531600B14601514601D146022805E7424
:10035600EB55324408FD7FB012010C22740C453275
:10036600FD7FB012010C227D2B7FB112010C227D84
:10037600077FB112010C22E531600B146015146081
:100386001D146022802774EE55324402FD7FB012A0
:10039600010C2274034532FD7FB012010C227D2B25
:1003A6007FB112010C227D077FB112010C228F331F
:1003B600798A77007D477FB112010C7DCB7FA2122F
:1003C600010C7DB27FCC12010CE53360077D0F7FF7
:1003D600B012010C228F34E53424FFB3E43324FF3A
:1003E600B3E433FA75F005A42477F9770075F005C0
:1003F600EAA42478F975F005EAA42479F975F005DC
:10040600EAA4247AF975F005EAA4247BF97D8274BE
:100416002F4534FF12010C7D8074224534FF1201F2
:100426000C7D30742C4534FF12010C7D0774324567
:1004360034FF12010C7D0774334534FF12010C2280
:100446008F358D36E53560267D037FB112010C7D33
:10045600017FA112010C7988E76004798E77017912
:100466008977007986E4F709F7798A770022798710
:10047600E536F719E4F722AC3774806F6033EF2462
:10048600FFB3E43324FFB3E433FA75F005A424770D
:10049600F9770175F005EAA4247AF9A70575F00540
:1004A600EAA42479F9A70375F005EAA4247BF9A741
:1004B60004228F388D397480653870030205DBE5B8
:1004C6003824FFB3E43324FFB3E43375F005A424E2
:1004D60078F97701E53824FFB3E43324FFB3E43336
:1004E60075F005A4247AF9E7FD74324538FF120148
:1004F6000CE53824FFB3E43324FFB3E43375F00589
:10050600A4247AF9E7FD74334538FF12010CE53867
:1005160024FFB3E43324FFB3E43375F005A4247950
:10052600F9E7600C7DE074224538FF12010C800A61
:100536007D8074224538FF12010CE53960167D2F47
:1005460074304538FF12010C7D2F74314538FF1287
:10055600010C80147D0374304538FF12010C7D03B5
:1005660074314538FF12010C7D01AF381202BCE52B
:100576003824FFB3E43324FFB3E43375F005A42431
:1005860079F9E7602AE53824FFB3E43324FFB3E4BE
:100596003375F005A4247BF9E7603A742C4538FFDF
:1005A6001201394480FD742C4538FF12010C227467
:1005B600224538FF1201394408FD74224538FF12DE
:1005C600010C742F4538FF1201394408FD742F457C
:1005D60038FF12010C228F3A7480653A70030206C6
:1005E60058E53A24FFB3E43324FFB3E43375F0054A
:1005F600A42478F97700742F453AFF12013954F78D
:10060600FD742F453AFF12010CE53A24FFB3E4339B
:1006160024FFB3E43375F005A42479F9E76029E5EE
:100626003A24FFB3E43324FFB3E43375F005A4247E
:100636007BF9E76013742C453AFF120139547FFDAC
:10064600742C453AFF12010C7D807422453AFF1244
:10065600010C228F3B7480653B6020E53B24FFB391
:10066600E43324FFB3E43375F005A42478F9E76096
:10067600031205DC7D01AF3B1202BC227FB11201E1
:1006860039F53C54027003020765798D7700743C96
:10069600553C700302070E24FC700302075A24F42B
:1006A600604624F0602424F060030207617D637FC6
:1006B600B112010C798A7707798B77FF0977FF7971
:1006C600897700798D7704020761798AE7FA6407EA
:1006D6006004EAB40807798A7706020761798977A0
:1006E60006798D7702020761798AE7FA6406600463
:1006F600EAB4070A798A7708798D7701805D798966
:10070600E7B40657770880537D037FB112010C7951
:100716008AE724F960051460068011798D770179DE
:100726008B770009772879887700802F798A770078
:100736007986E7094760247989E7601F7D017FA1F3
:1007460012010C798E7701798B77FF0977FF79890A
:10075600770080077D437FB112010C798F770122E4
:100766008F3D8C3E8D3F8A408B417FC1120139E51A
:100776003D24FFB3E43324FFB3E43375F005A4242A
:1007860079F98749754C40E53D23235403F54AE53D
:10079600412405F582E5403401F583E0F548E53D61
:1007A600B480028003020823754900754C20798FB6
:1007B600E7605AAF41AE4012020124F3504FAD4AF2
:1007C600AF41AE401202157D0CAF41AE401202158C
:1007D600E5412406F582E5403401F583E0FD04F0A9
:1007E600AF41AE401202157D09AF41AE401202156F
:1007F600754400E5442486F9E7FDAF41AE40120298
:10080600150544E54424F750EA798F7700740455BA
:1008160048600AE51C60061206825348FBE53F2441
:1008260004F582E53E3401F583E0600302090C74A9
:1008360020453DFF120139FA4548F5485410604DF0
:100846005348EFE5496034853F82853E83E0FAE50B
:100856003F2401F582E4353EF583E0C39A701C75AA
:1008660042007DFFAF3D12010C0542E54224C05017
:10087600F17D08AF3D1202BC02090CE53F2404F5E8
:1008860082E53E3401F583E54CF002090C7480657F
:100896003D6015E53F2407F582E53E3401F583E02A
:1008A600F404258C246F4023E53DB48059E53F24AC
:1008B60007F582E53E3401F583E0F404258CFB7AE6
:1008C60000EB24BFEA6480347D503BE53F2407F506
:1008D60082E53E3401F583E58CF07424453DFF1234
:1008E6000139F52AE53F2406F582E53E3401F58314
:1008F600E0F529853D287B6F7D747F5812023E7D89
:1009060001AF3D1202BCE53F2404F582E53E340109
:10091600F583E07003020E40853F82853E83E0FA50
:10092600E53F2401F582E4353EF583E0C39AF542BE
:1009360024FC4003020E407D03AF3FAE3E1201E9A8
:10094600FB7A00EB2404FBE43AFAAD427C00D3EBDD
:100956009DEA9C30D202B2E720E703020E40E53F53
:100966002407F582E53E3401F583E58CF0853F8268
:10097600853E83E0FA04F0E53F2402FDE4353EFCC3
:10098600ED2AF582E43CF583E0F54A853F82853E13
:1009960083E0FA04F0E53F2402FDE4353EFCED2A4F
:1009A600F582E43CF583E0F54B853F82853E83E0A6
:1009B600FA04F0E53F2402FDE4353EFCED2AF5821B
:1009C600E43CF583E0F54D853F82853E83E0FA04FD
:1009D600F0E53F2402FDE4353EFCED2AF582E43CD9
:1009E600F583E0F543E53F2406F582E53E3401F55F
:1009F60083E0FA654D600FE53F2406F582E53E3457
:100A060001F583E54DF0E53F2406F582E53E340128
:100A1600F583E004F0E54B603A14602724FE600D90
:100A260014603014601D24FE6003020CDDAF3D121D
:100A36000659E53F2404F582E53E3401F583E4F0EA
:100A4600020DEEE53F2404F582E53E3401F583E030
:100A56004480F0E53F2404F582E53E3401F583E069
:100A6600B4FF4FAD43AF3FAE3E1202367401654B45
:100A7600600AE54BB405028003020DEEE53F24044F
:100A8600F582E53E3401F583E0F52A854329853D67
:100A9600287B627D617F5812023EE53F2404F58281
:100AA600E53E3401F583E4F07D01AF3D1202BC0260
:100AB6000DEEE53DB480397FB1120139543CFA643C
:100AC60030602D7FB1120139C0E0AF3FAE3E12015A
:100AD600BDF52A798A8729D0028A287B317D447F11
:100AE6002112023EAD43AF3FAE3E120236020DEE7C
:100AF600E53F2404F582E53E3401F583E0547FF5B5
:100B060044E543C395445003854344853F82853E6F
:100B160083E0F54EE53F2402F552E4353EF551E516
:100B2600446014E552254EF582E43551F583E0FD27
:100B3600AF3D12010C054EC3E5449401F542602A0F
:100B4600E552254EF582E43551F583E0F550054E24
:100B5600901B3EF0907FE3741BF0907FE4743EF0B0
:100B6600907FE5E01542E54270D6853F82853E835B
:100B7600E54EF0E543C39544F543E53F2404F5828D
:100B8600E53E3401F583E0C39544F0E54370030286
:100B96000C2F853F82853E83E014F0FCE53F24025E
:100BA600FBE4353EFAEB2CF582E43AF583E543F0B7
:100BB600853F82853E83E014F0FCE53F2402FBE49A
:100BC600353EFAEB2CF582E43AF583E54DF0853FA8
:100BD60082853E83E014F0FCE53F2402FBE4353ECB
:100BE600FAEB2CF582E43AF583E54BF0853F8285F6
:100BF6003E83E014F0FCE53F2402FBE4353EFAEBCD
:100C06002CF582E43AF583E54AF0E53F2404F582C3
:100C1600E53E3401F583E0547FF0E53F2406F58296
:100C2600E53E3401F583E54DF07424453DFF1201A0
:100C360039F54254C06019E5496003020DEEE53FFF
:100C46002404F582E53E3401F58374FFF0020DEECF
:100C5600E53F2404F582E53E3401F583E06045E591
:100C66003F2404F582E53E3401F583E05480703478
:100C7600E53F2404F582E53E3401F583E070030286
:100C86000DEEE5497003020DEE853F82853E83E059
:100C9600FAE53F2401F582E4353EF583E0C39A6028
:100CA60003020DEE754208E5497014E53F2404F58C
:100CB60082E53E3401F583E05480600375420AAD57
:100CC60042AF3D1202BCE53F2404F582E53E340105
:100CD600F583E4F0020DEE75470075460075450094
:100CE600E543600B1543AF3FAE3E1201D0F545E537
:100CF60043600B1543AF3FAE3E1201D0F546E543C8
:100D0600600B1543AF3FAE3E1201D0F547E5436099
:100D16000D1543AF3FAE3E1201D0E54370F3E54BF0
:100D260024F6B40C004003020DDC901A67FA2A2A56
:100D360073751C00020DEE7D637FB112010C798B79
:100D4600770109779079887701020DEEE53F240453
:100D5600F582E53E3401F583E4F07D017FA11201C1
:100D66000C020DEEAB47AD46AF45120330020DEE59
:100D7600AD46AF45120446806F854737AB46AD4555
:100D8600AF3D12047D80617F001203DB7F401203BA
:100D9600DB805575F005E54AA42477F9770080488D
:100DA600AD45AF3D1204B8E53F2404F582E53E3477
:100DB60001F583E4F0E5412404F582E5403401F5CC
:100DC60083E4F05348EF8020AF3D1205DC8019AF75
:100DD6003D1206598012854D2A854B29853D287B73
:100DE600437D497F4912023EE53F2404F582E53EF4
:100DF6003401F583E06043853F82853E83E0FAE572
:100E06003F2401F582E4353EF583E0C39AF542249A
:100E1600FC50277D03AF3FAE3E1201E9FB7A00EBA3
:100E26002404FBE43AFAAD427C00D3EB9DEA9C3005
:100E3600D202B2E730E703020964E5412404F582F1
:100E4600E5403401F583E06003020EBF7420453DA2
:100E5600FF120139FA4548F54854C0605CE5412463
:100E660004F582E5403401F583E54CF0E54970462A
:100E76007425453DFF120139F542AA4C1A5AF5422E
:100E8600FAE5412404F582E5403401F583EAF07081
:100E96000FE5412404F582E5403401F583E54CF085
:100EA600748055486010E5412404F582E54034011C
:100EB600F583E04480F053483FE5412404F582E59C
:100EC600403401F583E07003021175E5412404F511
:100ED60082E5403401F583E0B4FF028003020F6C23
:100EE600AF41AE4012020124FC4003021175754267
:100EF60003E53DB48003754207AD4AAF41AE4012EB
:100F06000215AD42AF41AE40120215E5412406F589
:100F160082E5403401F583E0FD04F0AF41AE4012B6
:100F260002157D00AF41AE40120215E5412404F5DD
:100F360082E5403401F583E4F07427453DFF120154
:100F460039C0E0AF41AE40120201F52A853D28D0F6
:100F5600028A297B627D617F5212023E7D80AF3D0F
:100F66001202BC021175E549703AE5412404F58286
:100F7600E5403401F583E0548060297427453DFF40
:100F8600120139F54254F0FA64A060187480554293
:100F96006012E5412404F582E5403401F58374FFCF
:100FA600F0020E40E5412404F582E5403401F58364
:100FB600E0547FF544E5412401F582E43540F583AC
:100FC600E0854182854083FAE0C39A14FB7A00AD3E
:100FD600447C00ED2408FDE43CFCD3ED9BEC9A3008
:100FE600D202B2E720E703021175E544700302114D
:100FF60056E5412404F582E5403401F583E054804A
:101006006016E54424DF4010854443754201E53D02
:10101600B48013754205800E754320754200E53D88
:10102600B48003754204E5412401F582E43540F5B8
:1010360083E0FA04F0E5412402FDE43540FCED2AA4
:10104600F582E43CF583E54AF0E5412401F582E4C6
:101056003540F583E0FA04F0E5412402FDE435402D
:10106600FCED2AF582E43CF583E542F0E5412406F1
:10107600F582E5403401F583E0FA04F0E541240108
:10108600F582E43540F583E0FB04F0E5412402FDFA
:10109600E43540FCED2BF582E43CF583EAF0E541CE
:1010A6002401F582E43540F583E0FA04F0E54124B5
:1010B60002FDE43540FCED2AF582E43CF583E54388
:1010C600F0E5412401F582E43540F583E0F54FE58E
:1010D600412402F554E43540F553AF3D120139FA87
:1010E600E554254FF582E43553F583EAF0054FE5DF
:1010F60044C39543F544E5412404F582E5403401B3
:10110600F583E0C39543F01543E543602E907FE3F6
:10111600741BF0907FE4743EF0907FE5E542F0901A
:101126001B3EE0F542E554254FF582E43553F58341
:10113600E542F0054F1543E54370D2E5412401F53C
:1011460082E43540F583E54FF0E5446003020FF78E
:101156007D80AF3D1202BCE5412404F582E54034B2
:1011660001F583E4F0E53DB480028003020E40E51C
:10117600412405F582E5403401F583E548F0FAE5BA
:101186003F2405F582E53E3401F583EAF022E51BAE
:10119600B4FF4E538EF8438E01907F9C7430F090CE
:1011A6007F93F0907FE274D2F0907F957404F09074
:1011B6007F9E74FBF0907F9874B8F0907F98E0540F
:1011C600BFF0907F98E04408F0907F98E054DFF0FD
:1011D600751C007D0A7F861200237D0F7F77120023
:1011E60023E51BB44B07907F98E054F7F0E51BB45A
:1011F60001151202E97F001203B47F001203DB7FA0
:10120600401203DB751C01E51B60097F047E00129A
:101216000036151B227D007F0012010C907F98E09E
:1012260054F7F0907F98E054DFF0907F9CE4F090C4
:101236007F93F0907F98E054EFF0907F98E04440E1
:10124600F0751BFF228C558D568A578B5885568212
:10125600855583E0540260030212D2E5562401F557
:1012660082E43555F583E0F9EF2401F582E43EF595
:1012760083E0FA8F828E83FBE0C39B14FBE9D39B4A
:10128600504AAC02EF2402F55AE43EF559AD01E9A5
:101296006021855882855783E0FAE55A2CF582E469
:1012A6003559F583EAF00558E558700205570C1DC7
:1012B600ED70DFEF2401F582E43EF583ECF0E556B0
:1012C6002401F582E43555F5837440F0228E5B8F58
:1012D6005C8C5D8D5E8A5F8B60855E82855D83E05A
:1012E60054026003021370855C82855B83E0FAE535
:1012F6005C2401F582E4355BF583E0C39AF561244D
:10130600FC50677D03AF5CAE5B1201E92404F56215
:10131600D395615055855C82855B83E0F563E55C1A
:101326002402F565E4355BF564856261E562602358
:10133600E5652563F582E43564F583E0856082859D
:101346005F83F00560E5607002055F05631561E582
:101356006170DD855C82855B83E563F0E55E240173
:10136600F582E4355DF583E562F022907FD674065A
:10137600F0907F92E4F075890175881043D820902B
:101386007FA104F0907FE0E4F0907FE1F0907FDEB3
:10139600740FF0907FDFF0907F957404F0907F9E3D
:1013A60074FBF0907F9874B8F0756601E56625E0E9
:1013B600FA24C5F582E4347FF5837440F0E56625AA
:1013C600E0FA24B4F582E4347FF5837402F005660E
:1013D600E56624FC50D6756600AD667C007F087E07
:1013E6000112194F74202FF56E74203EF56D856E2F
:1013F60082856D83E4F0E56E2401F582E4356DF5B2
:1014060083E4F0E56E2402F582E56D3401F583E4AC
:10141600F0A3F0E56E2404F582E56D3401F583E46E
:10142600F0E56E2406F582E56D3401F583E4F0E51A
:101436006E2405F582E56D3401F5837410F00566BA
:10144600E56624FA509312121B7F00120167752A73
:10145600007529007528007B6B7D687F6312023E4C
:10146600752A4F752900907F92E0F5287B727D657D
:101476007F7612023E757302858C66051E757104B1
:101486007978E76003757106797DE760034371013A
:10149600AF71120167907FABE054106009907FAB8B
:1014A6007410F0021371907FABE054086014907FC3
:1014B600AB7408F07F0012016712121B438701020A
:1014C6001371907FABE05401700302186A757200C5
:1014D60075680074086568700302158E75F009E575
:1014E60072A42568901A8B93249B601A24FD605D74
:1014F60024FC603B24FE602624FB607424FB7003FE
:1015060002183102181374E82568F582E4347FF571
:1015160083E0F5675478700302183102184774E8BF
:101526002568F582E4347FF583E0F56B02183174A3
:10153600E82568F582E4347FF583E0FB7A00E4FD74
:10154600E56FFC4AF56FEB4DF57002183174E8252E
:1015560068F582E4347FF583E0FF7E007D0812198A
:1015660064E570FBE4FA4EF56FEF4BF57002183147
:1015760074E82568F582E4347FF583E0F56C24F899
:10158600400302183102184775F009E572A4256870
:10159600901A8B93F576901B0075F00E12192A029D
:1015A60018477480556760197407556725E0FA2453
:1015B600B4F582E4347FF583E0907F005401F08037
:1015C600177407556725E0FA24C4F582E4347FF5DD
:1015D60083E0907F005401F0907F01E4F0907FB5A6
:1015E6007402F002185E907F00E4F0907F01F090A4
:1015F6007FB57402F002185E747F55677003021897
:101606004774805567601F7407556725E0FA24B450
:10161600F582E4347FF5837401F074075567907F93
:10162600D74410F0801B7407556725E0FA24C4F5EB
:1016360082E4347FF5837401F0907FD7E567540721
:10164600F0907FD7E04420F0907FD7E054DFF0029F
:10165600185E747F5567700302184774805567607B
:10166600157407556725E0FA24B4F582E4347FF54E
:1016760083E4F002185E7407556725E0FA24C4F582
:1016860082E4347FF583E4F002185E756919756AA1
:1016960095907FD4E569F0907FD5E56AF002185EF3
:1016A600756919756AA7907FD4E569F0907FD5E5CD
:1016B6006AF002185EE56C25E02408F98769098757
:1016C6006AE56CB403607FFF7E0F1200D7FB7A00D9
:1016D600C002C0037FFE7E0F1200D7FF7E007D088A
:1016E600121964D0E02FFFD0E03EFEEF2400F56A29
:1016F600EE3401F569757400AB747A00E56A2BFF68
:10170600E5693AFE1200D7FA74002574F582E434CE
:101716007FF583EAF00574E57424EA50DB907FB523
:101726007416F002185E757500E56C25E02408F95C
:1017360087020987038B828A83E06039AB6AAA69CC
:10174600056ABBFF0205698B828A83E493FA7400FB
:101756002575F582E4347FF583EAF00575E56C2599
:10176600E02408F987020987038B828A83E0FAE579
:1017760075C39A40C7E56C25E02408F987020987F6
:10178600038B828A83E0907FB5F002185E907F001B
:10179600E519F0907FB57401F002185EE56B6008FC
:1017A600B401028003021847856B1902185E907F08
:1017B60000E51AF0907FB57401F002185EE56B60E3
:1017C60008B401028003021847856B1A02185E7F6F
:1017D600FF120167AD6BAF70AE6F1200A37F0012F0
:1017E6000167AF70AE6F1200D7FA656B606A805101
:1017F6007FFF120167AF70AE6F1200D7907F00F0C7
:10180600907FB57401F07F00120167804B75F00977
:10181600E572A42568901A8B93FA74E82568F58218
:10182600E4347FF583E0FBEAB5030B0568E568243D
:10183600F740030214D90572E57224F3400302143B
:10184600D6907FB47403F08015907F00E4F0907F0B
:1018560001F0907FB57402F0907FB47402F0907F2F
:10186600AB7401F07B807A7D7DBA7C7F7F487E25D4
:101876001212D37B407A7D7DCA7C7F7F407E241204
:10188600124BE51B6008121194858C6680637B40C1
:101896007A7E7DC67C7F7F207E2012124B7B287A43
:1018A600217D207C207F001207667B807A7E7DB6B4
:1018B6007C7F7F287E211212D37BC07A7D7DC87CF7
:1018C6007F7F307E2212124B7B387A237D307C223A
:1018D6007F401207667B007A7E7DB87C7F7F387EEC
:1018E600231212D37B487A257D407C247F80120701
:1018F60066C3E58C9566F566E573D39566501E75E9
:101906002A007529008566738566287B747D3E7F6F
:101916003E12023EE57324D05003757300858C6633
:041926000214812204
:10192A00CAC0E0E4936AA36009A3A3D5F0F5D0E0A6
:10193A00FA22E493FAA3E493F5828A83D0E0FAD0F8
:05194A00E0D0E0E473B1
:10194F00C0F0ED8FF0A4CFC5F0CCA42CCE8DF0A4B9
:05195F002EFED0F02275
:10196400ED540F600AFDC3EF33FFEE33FEDDF722C3
:0E197400E493F608A3EFB582F7EEB583F322F5
:00000001FF
